:020000040000FA
:020000000528D1
:08000800090083128501073095
:1000100099008316850185140000851530309F00F6
:100020009F148C010C1783120B1705309F00A10140
:10003000A201A3015E2054206420742044202008E3
:100040008B3C03182B284D200130A2000130A30067
:100050007D207D201C282008873C03183928A20811
:10006000031D1C28A30803191C284F204B207420B3
:100070001C284B20A20120087A3C031C1C280130BC
:10008000A100562058201C280C139F146300000068
:100090001E08A000080005100800051408004B20E9
:1000A00077204D207D200800051508000511080067
:1000B0005A20080005160800051208005A207D2065
:1000C0007D207D205C20080085190800742085199A
:1000D00008004B20442020087A3C03181C28A1016A
:1000E0005C205420742008000130A40080280530D2
:1000F000A40080280A30A40080283230A400802880
:080100008128A40B80280800EF
:084000000000010000000000B7
:02400E00863FEB
:00000001FF
